:100000000C9473010C94A0070C9476070C944C0785
:100010000C9422070C94F8060C94CE060C94A401C0
:100020000C94A4010C94A4010C94A4010C94A401BC
:100030000C94A4010C94A4010C94A4010C94A401AC
:100040000C94A4010C94A4010C94A4010C94A4019C
:100050000C94A4010C94A4010C94A4010C948406A7
:100060000C94A4010C944E060C9424060C94A40148
:100070000C94A4010C94A4010C94A4010C94A4016C
:100080000C94A4010C94A4010C94A4010C94A4015C
:100090000C94A4010C94A4010C94A4010C94A4014C
:1000A0000C94A4010C94A4010C94A4010C94A4013C
:1000B0000C94A4010C94A4010C94A4010C94A4012C
:1000C0000C94A4010C94A4010C94A4010C94A4011C
:1000D0000C94A4010C94A4010C94A4010C94A4010C
:1000E0000C94A4010C9407030C94A6010C944602F2
:1000F0000C94F2020C94EC010C94EC020C94CA07E0
:100100000C94F6020C9431030C940E020C94FE0233
:100110000C9401030C940B030C9427030C94190307
:100120000C9400020C94AE020C942C030C94230447
:100130000C949D0B0C9423030C94DD010C941F0371
:100140000C94FA020C9411030C9415030C941F04E4
:100150000C942D032F0A002300230023005C23238B
:1001600023235265616C53696D47656172230000FA
:100170000020002300260029002C002F0032000060
:1001800001000003010601090100002100240027ED
:10019000002A002D00300033000101000004010797
:1001A000010A0100002200250028002B002E00314A
:1001B00000340002010000050108010B01050505DE
:1001C00005070508080808020202020A0A080804CE
:1001D00004040401010101010101010303030303FC
:1001E000030303040707070C0C0C0C0C0C0C0C028B
:1001F00002020206060606060606060B0B0B0B0B92
:100200000B0B0B010210202008081020401020408A
:1002100080020102010804020101020408102040CA
:1002200080804020100804020180040201804020E8
:100230001008040201080402010102040810204011
:1002400080010204081020408000000A0B02090C03
:100250000D0E08070304010000000000000000006C
:10026000000000000000000000000000000000008E
:10027000000000000012111000000000000000004B
:100280000000000000000000000000000000002F3F
:100290000A002300230023005C23232323526561EB
:1002A0006C53696D4765617223000A000A003D00C6
:1002B0000A003D003D300A002E4F46460A003D31FF
:1002C0000A002E4F4E0A002F0A00230023002300AD
:1002D0005C232323235265616C53696D476561720A
:1002E0002300CA079D0B11241FBECFEFD1E2DEBF52
:1002F000CDBF00E00CBF29E0A8E3B5E001C01D922E
:10030000A133B207E1F715E0A0E0B2E0E0E9FCE1DB
:1003100000E00BBF02C007900D92A833B107D9F7D8
:1003200011E0C2E7D1E000E006C021970109802F6B
:10033000FE010E94F10BC137D10780E00807A9F741
:100340000E9462080C94360E0C940000AF92BF928B
:10035000CF92DF92EF92FF920F931F93CF93DF9391
:100360006C017B018B01040F151FEB015E01AE18C0
:10037000BF08C017D10759F06991D601ED91FC91E2
:100380000190F081E02DC6011995892B79F7C501FF
:10039000DF91CF911F910F91FF90EF90DF90CF9061
:1003A000BF90AF900895E7E5F6E044815581608104
:1003B00071818BEA95E00C94A601FC01538D448D6C
:1003C000252F30E0842F90E0821B930B541710F000
:1003D000CF96089501970895FC01918D828D98170D
:1003E00061F0A28DAE0FBF2FB11D5D968C91928DE5
:1003F0009F5F9F73928F90E008958FEF9FEF089516
:10040000FC01918D828D981731F0828DE80FF11DDE
:10041000858D90E008958FEF9FEF0895FC01918DF9
:10042000228D892F90E0805C9F4F821B91098F73F2
:10043000992708958BEA95E00E940E0221E0892B0E
:1004400009F420E0822F0895FC01A48DA80FB92F94
:10045000B11DA35ABF4F2C91848D90E001968F73EC
:100460009927848FA689B7892C93A089B1898C910B
:10047000837080648C93938D848D981306C002885A
:10048000F389E02D80818F7D80830895EF92FF9224
:100490000F931F93CF93DF93EC0181E0888F9B8DA7
:1004A0008C8D98131AC0E889F989808185FF15C061
:1004B0009FB7F894EE89FF896083E889F989808184
:1004C0008370806480839FBF81E090E0DF91CF9153
:1004D0001F910F91FF90EF900895F62E0B8D10E075
:1004E0000F5F1F4F0F731127E02E8C8D8E110CC0E4
:1004F0000FB607FCFACFE889F989808185FFF5CF2F
:10050000CE010E942402F1CFEB8DEC0FFD2FF11DE7
:10051000E35AFF4FF0829FB7F8940B8FEA89FB896B
:1005200080818062CFCF0F931F93CF93DF938C0195
:10053000D0E0C0E0F801EC0FFD1F6491662341F0AC
:100540008BEA95E00E944602892B11F02196F2CFAA
:10055000CE01DF91CF911F910F910895CF93DF933B
:10056000EC01888D8823B9F0AA89BB89E889F989CB
:100570008C9185FD03C0808186FD0DC00FB607FC00
:10058000F7CF8C9185FFF2CF808185FFEDCFCE0133
:100590000E942402E9CFDF91CF91089581508231EA
:1005A00008F05AC0E82FF0E08827E652FD4F8F4F41
:1005B0000C94F10BFA02FE02EC02F202F6022C039A
:1005C000010307030B031103150319031F0323037F
:1005D0002C0327032D033103809180008F778093B4
:1005E00080000895809180008F7DF9CF80918000F8
:1005F000877FF5CF84B58F7784BD089584B58F7DCF
:10060000FBCF8091B0008F778093B00008958091E8
:10061000B0008F7DF9CF809190008F77809390000C
:100620000895809190008F7DF9CF80919000877F11
:10063000F5CF8091A0008F778093A00008958091DE
:10064000A0008F7DF9CF8091A000877FF5CF8091AA
:1006500020018F77809320010895809120018F7D64
:10066000F9CF80912001877FF5CF1F93CF93DF9340
:10067000282F30E0F901E75BFD4F8491F901ED5F30
:10068000FD4FD491F901E354FE4FC491CC23A9F05E
:10069000162F81110E94CE02EC2FF0E0EE0FFF1F0B
:1006A000ED55FE4FA591B4918FB7F894EC911111CF
:1006B00008C0D095DE23DC938FBFDF91CF911F91CF
:1006C0000895DE2BF8CFCF93DF9390E0FC01ED5F30
:1006D000FD4F249183549E4FFC0184918823C9F0DF
:1006E00090E0880F991FFC01E757FE4FA591B49148
:1006F000FC01ED55FE4FC591D49161110DC09FB71E
:10070000F8948C91209582238C93888128232883C8
:100710009FBFDF91CF910895623051F49FB7F89455
:100720003C91822F809583238C93E8812E2BEFCFF1
:100730008FB7F894EC912E2B2C938FBFEACF863392
:1007400008F0865320917B00982F9870277F922B7A
:1007500090937B008770806480937C0080917A0006
:10076000806480937A0080917A0086FDFCCF80912E
:1007700078009091790008953FB7F8948091A3058F
:100780009091A405A091A505B091A60526B5A89BBA
:1007900005C02F3F19F00196A11DB11D3FBFBA2F13
:1007A000A92F982F8827BC01CD01620F711D811DD3
:1007B000911D42E0660F771F881F991F4A95D1F758
:1007C00008958F929F92AF92BF92CF92DF92EF9255
:1007D000FF924B015C010E94BC036B017C010E94F3
:1007E000BC036C197D098E099F09683E7340810521
:1007F0009105A8F321E0821A9108A108B10888EEBA
:10080000C80E83E0D81EE11CF11C81149104A104E0
:10081000B10429F7FF90EF90DF90CF90BF90AF9099
:100820009F908F9008952FB7F89460919F057091D5
:10083000A0058091A1059091A2052FBF0895862F54
:10084000642F0C946303CF93DF93FC01218930E084
:10085000F901E75BFD4F8491F901ED5FFD4FD49104
:10086000F901E354FE4FC491CC2379F081110E9429
:10087000CE02EC2FF0E0EE0FFF1FE159FE4FA591E5
:10088000B491EC91ED2381E009F480E08170DF9177
:10089000CF910895DC01ED91FD918081ED91FD9165
:1008A0009081ED91FD916C9163708E2309F06460ED
:1008B0009F2309F06860E7E6F4E0E60FF11D659517
:1008C00065956D936D917D918D919D91099423C056
:1008D0001AC012C016C010C01EC009C014C013C078
:1008E00006C019C009C00DC007C00DC014C06250B9
:1008F0007040804090400BC06150704080409040FC
:1009000006C06E5F01C06F5F7F4F8F4F9F4F9E93FA
:100910008E937E936E9308958F929F92AF92BF9223
:100920000F931F93CF93DF93CDB7DEB7A1970FB689
:10093000F894DEBF0FBECDBF19A2423008F44AE0E2
:100940008E010F5D1F4F842E912CB12CA12CA5017F
:1009500094010E94CF0BE62FB901CA01EA3044F599
:10096000E05DD801EE938D01232B242B252B79F705
:1009700090E080E0109769F0FD0101900020E9F718
:100980003197AF014A1B5B0BBD018BEA95E00E94DA
:10099000A601A1960FB6F894DEBF0FBECDBFDF91C2
:1009A000CF911F910F91BF90AF909F908F9008951E
:1009B000E95CD7CFCF92DF92EF92FF92CF93DF9394
:1009C0006C01990FEE08FF08F7FE19C06DE28BEA83
:1009D00095E00E944602EC0166277727CB016C194F
:1009E0007D098E099F094AE00E948C048C0F9D1F8F
:1009F000DF91CF91FF90EF90DF90CF9008954AE084
:100A0000C701B601DF91CF91FF90EF90DF90CF90BB
:100A10000C948C04009769F0FC0101900020E9F728
:100A20003197AF01481B590BBC018BEA95E00C9440
:100A3000A60190E080E008958BEA95E00E940E0206
:100A4000892B09F457C08BEA95E00E94EC018C37A2
:100A500019F58DE591E00E9493028EEC92E00E94E0
:100A60000A058BE591E00E94930287E090E00E94E6
:100A7000DA0489E591E00E94930284E092E00E940A
:100A80000A0587E591E00E9493020E94D30184E564
:100A900091E00E949302D0CF8C3329F410929D05EF
:100AA00010929C05C9CF8A3099F48091380560E096
:100AB000813309F461E08EE10E94350380913905AC
:100AC00060E0813309F461E084E10E943503E6CF00
:100AD00020919C0530919D0524363105FCF6F901E5
:100AE000E85CFA4F80832F5F3F4F30939D05209342
:100AF0009C05A2CF08950E941A0281110E941C0534
:100B000080E090E0892B49F080E090E0892B29F08B
:100B10000E94000081110E94000080E090E0892B7B
:100B200049F080E090E0892B29F00E9400008111BB
:100B30000E94000080E090E0892B49F080E090E086
:100B4000892B29F00E94000081110C940000089567
:100B50000E94FF0D0F931F93CF93DF93EC018881C9
:100B60009981009759F02A813B812617370730F089
:100B700081E0DF91CF911F910F9108958B016F5FFD
:100B80007F4F0E941E0D009759F0998388831B8325
:100B90000A832C813D81232B59F7FC011082E8CF79
:100BA00080E0E7CFCF93DF93EC01888199810097B4
:100BB00011F00E94950C198218821D821C821B82E2
:100BC0001A82DF91CF910895EF92FF920F931F93B6
:100BD000CF93DF93EC017B018A01BA010E94AA0541
:100BE00081110BC0CE010E94D205CE01DF91CF91C1
:100BF0001F910F91FF90EF9008951D830C83B70113
:100C0000888199810E94150EF0CFCF93DF93EC017C
:100C1000FB018617970749F06081718161157105A5
:100C200041F0448155810E94E405CE01DF91CF91CE
:100C300008950E94D205F9CFFC018081918100972F
:100C400011F00C94950C08951F920F920FB60F920D
:100C500011240BB60F922F933F934F935F936F9393
:100C60007F938F939F93AF93BF93EF93FF938BEA01
:100C700095E00E942402FF91EF91BF91AF919F9167
:100C80008F917F916F915F914F913F912F910F9035
:100C90000BBE0F900FBE0F901F9018951F920F92D2
:100CA0000FB60F9211240BB60F922F938F939F9331
:100CB000EF93FF93E091BB05F091BC058081E0913B
:100CC000C105F091C20582FD1DC090818091C405CF
:100CD0008F5F8F732091C505821741F0E091C405A5
:100CE000F0E0E555FA4F958F8093C405FF91EF91A1
:100CF0009F918F912F910F900BBE0F900FBE0F9071
:100D00001F9018958081F2CF1F920F920FB60F920D
:100D100011242F933F938F939F93AF93BF93809111
:100D20009F059091A005A091A105B091A2053091D9
:100D30009E0523E0230F2D3758F50196A11DB11D07
:100D400020939E0580939F059093A005A093A105F5
:100D5000B093A2058091A3059091A405A091A5054B
:100D6000B091A6050196A11DB11D8093A305909396
:100D7000A405A093A505B093A605BF91AF919F913F
:100D80008F913F912F910F900FBE0F901F9018954C
:100D900026E8230F0296A11DB11DD2CF1F920F92FC
:100DA0000FB60F9211240BB60F922F933F934F93D0
:100DB0005F936F937F938F939F93AF93BF93EF93C3
:100DC000FF9390E080E00E944A04FF91EF91BF9171
:100DD000AF919F918F917F916F915F914F913F91D3
:100DE0002F910F900BBE0F900FBE0F901F90189574
:100DF0001F920F920FB60F9211240BB60F922F93E2
:100E00003F934F935F936F937F938F939F93AF9392
:100E1000BF93EF93FF9390E080E00E944A04FF911C
:100E2000EF91BF91AF919F918F917F916F915F9162
:100E30004F913F912F910F900BBE0F900FBE0F90CF
:100E40001F9018951F920F920FB60F9211240BB698
:100E50000F922F933F934F935F936F937F938F9353
:100E60009F93AF93BF93EF93FF9390E080E00E9436
:100E70004A04FF91EF91BF91AF919F918F917F9124
:100E80006F915F914F913F912F910F900BBE0F90FB
:100E90000FBE0F901F9018951F920F920FB60F92D2
:100EA00011240BB60F922F933F934F935F936F9341
:100EB0007F938F939F93AF93BF93EF93FF9390E0B4
:100EC00080E00E944A04FF91EF91BF91AF919F9102
:100ED0008F917F916F915F914F913F912F910F90E3
:100EE0000BBE0F900FBE0F901F9018951F920F9280
:100EF0000FB60F9211240BB60F922F933F934F937F
:100F00005F936F937F938F939F93AF93BF93EF9371
:100F1000FF9390E080E00E944A04FF91EF91BF911F
:100F2000AF919F918F917F916F915F914F913F9181
:100F30002F910F900BBE0F900FBE0F901F90189522
:100F40001F920F920FB60F9211240BB60F922F9390
:100F50003F934F935F936F937F938F939F93AF9341
:100F6000BF93EF93FF9390E080E00E944A04FF91CB
:100F7000EF91BF91AF919F918F917F916F915F9111
:100F80004F913F912F910F900BBE0F900FBE0F907E
:100F90001F9018951092AE051092AD0588EE93E063
:100FA000A0E0B0E08093AF059093B005A093B105A9
:100FB000B093B20588EB92E09093AC058093AB05BB
:100FC00085EC90E09093B8058093B70584EC90E0B1
:100FD0009093BA058093B90580EC90E09093BC059E
:100FE0008093BB0581EC90E09093BE058093BD0596
:100FF00082EC90E09093C0058093BF0586EC90E072
:101000009093C2058093C1051092C4051092C50546
:101010001092C6051092C705A8E4B6E090E080E003
:1010200041E2FC013E9621E030E08630910510F46B
:1010300030E020E0E20FF31F40935700E491ED937E
:1010400001968930910569F7EDE5F6E08DE299E0CA
:101050004AE050E02AEC32E01282138214821582B8
:1010600057834683108631832083118A72968E17A8
:101070009F0791F7109258061092570610925A0641
:101080001092590610925C0610925B0650E040E008
:101090006EEE72E087E596E00E94E405109252063B
:1010A0001092510610925406109253061092560652
:1010B000109255064DE050E061EE72E081E596E059
:1010C0000C94E405CF93DF93CDB7DEB72F970FB61F
:1010D000F894DEBF0FBECDBF789484B5826084BD26
:1010E00084B5816084BD85B5826085BD85B581602C
:1010F00085BD80916E00816080936E0010928100AA
:101100008091810082608093810080918100816064
:101110008093810080918000816080938000809125
:10112000B10084608093B1008091B00081608093B1
:10113000B000809191008260809391008091910035
:1011400081608093910080919000816080939000F5
:101150008091A10082608093A1008091A1008160B4
:101160008093A1008091A00081608093A000809175
:10117000210182608093210180912101816080930F
:1011800021018091200181608093200180917A006B
:10119000846080937A0080917A00826080937A00E4
:1011A00080917A00816080937A0080917A008068D3
:1011B00080937A001092C100E091BB05F091BC05CC
:1011C00082E08083E091B705F091B8051082E0914C
:1011D000B905F091BA0580E180831092C305E091D2
:1011E000BF05F091C00586E08083E091BD05F091D8
:1011F000BE05808180618083E091BD05F091BE05D0
:10120000808188608083E091BD05F091BE0580817A
:1012100080688083E091BD05F091BE0580818F7D5F
:10122000808382E390E0A0E0B0E08093AF059093EC
:10123000B005A093B105B093B20568EE73E080E00D
:1012400090E00E94E10349E4E42E46E0F42E51E5EB
:10125000C52E56E0D52E8E010F5F1F4FD7018D9101
:101260007D011B861A861D861C861F861E8640E110
:10127000B80190E00E94A50BF80101900020E9F769
:101280003197AF01401B510BB801CE010A960E9465
:10129000E4051A8219821C821B821E821D8267E568
:1012A00076E0C8010E9405068E859F858A849B840E
:1012B000AD80BE80A80EB91E81149104B9F1892BAE
:1012C00089F0B501C8010E94AA05882379F1298116
:1012D0003A818D819E81B401820F931F0E94150E69
:1012E000BE82AD82B80187E596E00E940506C8017E
:1012F0000E941C06CE010A960E941C06CE14DF0432
:1013000009F0ACCF00915706109158060115110550
:1013100089F0F8018081882369F0082E000C990B70
:101320000E94040ED8018D938D01F3CFC8010E9455
:10133000D205D8CF88E992E00E9493028EEC92E029
:101340000E940A0586E992E00E94930287E090E0FD
:101350000E94DA0484E992E00E94930284E092E021
:101360000E940A0582E992E00E9493020E94D30142
:101370008FE892E00E9493029DE2C92E99E0D92E57
:101380002DE5E22E26E0F22E04E112E03AE0A32E53
:10139000B12CF80190807181D701ED91FC91028010
:1013A000F381E02D42E050E0692DC7011995F70166
:1013B000918A10860190F081E02D0190F081E02D5E
:1013C000C7011995882339F0D70118968C91189781
:1013D000836018968C930E941304F70162837383D1
:1013E00084839583B782A6820C5F1F4FF2E1EF0ED4
:1013F000F11CCE14DF0469F661E08EE10E94630304
:1014000061E08EE10E94350361E084E10E946303A4
:1014100061E084E10E94350368EB7BE080E090E0CE
:101420000E94E10360E08EE10E94350360E084E108
:101430000E9435030E9413044B015C0180910A0253
:1014400090910B02A0910C02B0910D02AC01BD0174
:101450004854544F6F4F7F4F84169506A606B70623
:1014600028F488169906AA06BB0690F580ED92E04E
:101470000E9493028EEC92E00E940A058EEC92E0AC
:101480000E94930287E090E00E94DA048CEC92E0E4
:101490000E94930284E092E00E940A058AEC92E0A6
:1014A0000E9493020E94D30187EC92E00E94930273
:1014B00080920A0290920B02A0920C02B0920D024E
:1014C0008092000290920102A0920202B092030266
:1014D00061E070E080E090E00E94E10384E1682E2A
:1014E00082E0782E0DE516E0D80118968C911897B9
:1014F0008B7F18968C931897ED91FC910190F08159
:10150000E02DC8011995D82EF80180858695817047
:10151000D81609F4AAC00E941304D80112966D933C
:101520007D938D939C93159718968C91B2E08B27A1
:10153000F8018087D80118969C91892F847090FDBE
:10154000E2C0882391F0F301C280D38064E275E0A9
:10155000C6010E941C0E892B09F4CFC0C6010E944F
:101560000A0582EC92E00E9493020E5E1F4FB4E0E7
:101570006B0E711C0E151F0509F0B6CF86E30E9495
:101580009F038C018091A9059091AA059C012F5081
:1015900031090217130724F00F9680179107B4F44E
:1015A0000B3011059CF01093AA050093A9058FEE4E
:1015B00092E00E940A0582EB92E00E949302C80129
:1015C0000E94DA0480EB92E00E94930287E30E947B
:1015D0009F038C018091A7059091A8059C012F5035
:1015E00031090217130724F00F9680179107B4F4FE
:1015F0000B3011059CF01093A8050093A70589EF07
:1016000092E00E940A058EEA92E00E949302C801CD
:101610000E94DA048CEA92E00E9493028091000218
:1016200090910102A0910202B0910302AC01BD01B0
:101630004C595F4F6F4F7F4F84169506A606B7062D
:1016400028F488169906AA06BB0660F48AEA92E096
:101650000E9493028092000290920102A0920202E4
:10166000B09203020E947B05E5CE0E941304D801CC
:1016700012962D913D914D915C9115971B012C0176
:10168000221A330A440A550AB201A10116968D9115
:101690009C91B0E0A0E0481759076A077B0708F45F
:1016A00049CFD80118968C918170D81609F442CF91
:1016B0000E941304F8016283738384839583808579
:1016C000F1E08F278460D80118968C930E94130450
:1016D000F8012185328543855485621B730B840B89
:1016E000950B658776878787908B0E941304F80196
:1016F00061877287838794871DCFC6010E940A0580
:101700008EEB92E030CF882309F42FCFD3011296CD
:10171000CD90DC9064E275E0C6010E941C0E892B1E
:1017200031F0C6010E940A0588EB92E01CCFC60189
:101730000E940A0584EB92E016CF81E596E00E94B4
:101740001C0687E596E00C941C06BB27FB01552779
:10175000AA27880F991FAA1FA41710F0A41B83950E
:101760005051B9F7A05DAA3308F0A95DA193009785
:1017700079F7B111B1931192CB010C94BF0BDC013D
:10178000FC01672F71917723E1F7329704C07C91B8
:101790006D9370836291AE17BF07C8F30895A1E2FD
:1017A0001A2EAA1BBB1BFD010DC0AA1FBB1FEE1FDB
:1017B000FF1FA217B307E407F50720F0A21BB30B26
:1017C000E40BF50B661F771F881F991F1A9469F7A2
:1017D00060957095809590959B01AC01BD01CF01FE
:1017E0000895EE0FFF1F881F8BBF0790F691E02D25
:1017F00019940F931F93CF93DF938230910510F4C8
:1018000082E090E0E0912F09F091300930E020E093
:10181000B0E0A0E0309799F42115310509F44AC0F1
:10182000281B390B24303105D8F58A819B8161153D
:10183000710589F1FB0193838283FE0111C0408110
:1018400051810281138148175907E0F04817590761
:1018500099F4109761F012960C93129713961C93BB
:101860003296CF01DF91CF911F910F910895009390
:101870002F0910933009F4CF2115310551F042178B
:10188000530738F0A901DB019A01BD01DF01F8011E
:10189000C1CFEF01F9CF9093300980932F09CDCFBD
:1018A000FE01E20FF31F8193919322503109398396
:1018B0002883D7CF20912D0930912E09232B41F475
:1018C000209110023091110230932E0920932D099E
:1018D00020910E0230910F022115310541F42DB7F0
:1018E0003EB74091120250911302241B350BE09138
:1018F0002D09F0912E09E217F307A0F42E1B3F0BE0
:101900002817390778F0AC014E5F5F4F2417350771
:1019100048F04E0F5F1F50932E0940932D0981937D
:1019200091939FCFF0E0E0E09CCFCF93DF930097BF
:10193000E9F0FC01329713821282A0912F09B09135
:101940003009ED0130E020E01097A1F420813181D1
:10195000820F931F20912D0930912E0928173907E6
:1019600009F061C0F0932E09E0932D09DF91CF912A
:101970000895EA01CE17DF07E8F54A815B819E01F1
:1019800041155105B1F7E901FB83EA83499159916A
:10199000C40FD51FEC17FD0761F480819181029679
:1019A000840F951FE90199838883828193819B83AA
:1019B0008A83F0E0E0E012968D919C911397009756
:1019C000B9F52D913C911197CD010296820F931F8D
:1019D00020912D0930912E092817390739F63097B3
:1019E00051F51092300910922F09B0932E09A0934F
:1019F0002D09BCCFD383C28340815181840F951FB1
:101A0000C817D90761F44E5F5F4F88819981480FED
:101A1000591F518340838A819B819383828321153F
:101A2000310509F0B0CFF0933009E0932F099ECF34
:101A3000FD01DC01C0CF13821282D7CF4F925F929B
:101A40006F927F928F929F92AF92BF92CF92DF92CE
:101A5000EF92FF920F931F93CF93DF938C01009728
:101A600099F4CB01DF91CF911F910F91FF90EF90EF
:101A7000DF90CF90BF90AF909F908F907F906F90AE
:101A80005F904F900C94F90BFC01E60FF71F9C013F
:101A900022503109E217F30708F4AEC0D901CD9105
:101AA000DC911197C617D70720F1C530D10578F022
:101AB000CE0104978617970750F0C61BD70B2297C5
:101AC000C193D1936D937C93CF010E94950CC80173
:101AD000DF91CF911F910F91FF90EF90DF90CF900A
:101AE000BF90AF909F908F907F906F905F904F903E
:101AF00008955B01AC1ABD0A4C018C0E9D1EA0918D
:101B00002F09B0913009512C412CF12CE12C109768
:101B100031F580912D0990912E098815990509F0CC
:101B20005CC04616570608F058C080910E0290918E
:101B30000F02009741F48DB79EB740911202509169
:101B40001302841B950BE817F90708F055C0F093B2
:101B50002E09E0932D09F90171836083B8CF8D912F
:101B60009C91119712966C90129713967C901397F4
:101B7000A815B90559F56C0142E0C40ED11CCA1470
:101B8000DB0420F1AC014A195B09DA0112961597C2
:101B900080F06282738251834083D9016D937C937C
:101BA000E114F10471F0D7011396FC93EE931297B0
:101BB0008ECF22968C0F9D1FF90191838083F301B4
:101BC000EFCFF0933009E0932F0981CF48165906E3
:101BD00008F42C017D01D3019ACFCB010E94F90BAF
:101BE0007C01009749F0AE01B8010E940C0EC801BB
:101BF0000E94950C87016BCF10E000E068CF81E078
:101C000090E0F8940C94360E9111089581568A5103
:101C100008F4805285580895FB01DC0102C0019050
:101C20000D9241505040D8F70895FB01DC0101901E
:101C30000D920020E1F70895FB0151915523A9F081
:101C4000BF01DC014D9145174111E1F759F4CD0178
:101C50000190002049F04D9140154111C9F3FB015D
:101C60004111EFCF81E090E00197089511E0C2E7C4
:101C7000D1E000E006C0802FFE010E94F10B21960A
:101C8000011DC337D10780E00807A9F7F894FFCFFB
:101C9000FFFFFFFF332E322E3400FFFFFFFF000057
:101CA000310980002D0003032E0013032C002303B1
:101CB0002B002F032A003903290046032800530371
:101CC00027005F032600690325007C0307008F03BC
:101CD0000F00A0030A00AA031F00B5031500C803E4
:101CE0002300DB032400EB032200FB032100080494
:101CF000100015041200210411002D040E003F04F1
:101D00000C00510419005D040B00690408007704FD
:101D100009008504060092042F009F043000AC04E3
:101D20003100BC043200CB043300D8043400E60494
:101D30003500F404030004050200100505001C052D
:101D400004002805000000004602A601DD01AE02E5
:101D50000E02EC0100020000000023041F044D39B4
:101D60004176696174696F6E2D54424D2D504E4C11
:101D7000003735364536423737363939393900502C
:101D80004F545F50414E454C00504F545F425241BA
:101D90004B450053575F4C44475F4C545F444E2EB5
:101DA00053570053575F4C44475F4C545F55502E78
:101DB00053570053575F50554C53452E53570053BC
:101DC000575F4E41562E53570053575F5354524F4F
:101DD00042452E53570053575F44494D4D45522EAF
:101DE00053570053575F434142494E2E53570053B8
:101DF000575F4143434553530042544E5F4D414961
:101E00004E5F47454E5F52455345540042544E5F26
:101E1000535442595F47454E5F5245534554005312
:101E2000575F4D41494E5F504F5745522E53570013
:101E300042544E5F53484946540053575F465545F8
:101E40004C2E53570042544E5F4D41535445525F00
:101E50005741524E494E470042544E5F4D415354F4
:101E600045525F43415554494F4E0053575F534FBE
:101E7000555243455F444E2E53570053575F534FBF
:101E8000555243455F55502E53570053575F4745B2
:101E90004E5F444E2E53570053575F47454E5F5594
:101EA000502E53570053575F53544152545F444E82
:101EB0000053575F53544152545F55500053575F7E
:101EC00049474E4954494F4E5F444E2E5357005395
:101ED000575F49474E4954494F4E5F55502E53570F
:101EE0000053575F42505F444E2E53570053575F85
:101EF00042505F55502E53570053575F5452494D2F
:101F00005F444E2E53570053575F5452494D5F550F
:101F1000502E53570053575F454C545F444E2E5339
:101F2000570053575F454C545F55502E535700533D
:101F3000575F41465F4943452E53570053575F490A
:101F400043455F4C494748542E53570053575F5001
:101F5000524F505F4943452E53570053575F5753D5
:101F60005F4943452E53570053575F5049544F54D0
:101F70005F4C2E53570053575F5049544F545F5294
:101F80002E53570053575F494E4552545F534550A7
:101F90002E53570053575F41435F444E2E53570013
:101FA00053575F41435F55502E53570053575F427D
:101FB0004C4545442E53570053575F505245535399
:081FC0005552452E5357000055
:00000001FF
